:1000000096C0AFC0AEC0ADC0ACC034C2AAC0A9C01B
:10001000A8C0A7C0A6C0A5C0A4C0A3C0A2C0A1C0BC
:10002000A0C09FC09EC0E8C5E9C5EAC5EBC5ECC548
:10003000EBC5EAC5E9C5EBC5FAC503C614C604C6D7
:1000400006C60AC60EC624C626C640C642C644C652
:1000500043C642C641C644C6A0C64CC69EC64DC68F
:100060004EC65BC65EC699C698C697C696C695C666
:1000700094C693C692C691C690C68FC68EC68DC6CC
:100080008CC68BC68AC687C612011001FF00000805
:10009000C016B30620460102000134035500530088
:1000A000420032004C005000540020006C006F00F1
:1000B00077002D007300700065006500640020006B
:1000C0006100640061007000740065007200240328
:1000D00068006100660074006D0061006E006E00D3
:1000E000230073006F0066007400770061007200E7
:1000F0006500040309040902370001010080320988
:1001000004000002FF0000000705010208000007CC
:100110000581020800000904000102FF0000000739
:1001200005010308000A0705810308000A001124DD
:100130001FBECFE5D4E0DEBFCDBF10E0A0E6B0E04B
:10014000E8E6FFE002C005900D92A436B107D9F7AA
:1001500010E0A4E6B0E001C01D92AD3CB107E1F7AC
:1001600034C64ECFCF93DC01C62F809160008E3114
:10017000F1F08091600084FF07C08091A20098E8B0
:1001800089278093A20003C08AE580936000E3EA98
:10019000F0E09C2F91509F3F19F08D918193FACF01
:1001A0006C2F83EA90E062D1CC5FC0936000CF9166
:1001B0000895FF920F931F93CF93DF936091B30045
:1001C00016160CF0CBC08091AF00C3ECD0E0C81B7A
:1001D000D109162F135000E090E8F92E8091AE005F
:1001E0008D3211F48AEFD0D38091AE008F3F21F48D
:1001F000612FCE01D1D4ACC08D3209F092C03AE566
:1002000030936100183009F09FC02881822F8076DA
:1002100009F075C0E0EAF0E00093A000998199230D
:1002200089F42F71223059F48C81813841F4902F58
:10023000809160008E3109F491E09093A0001182CA
:1002400002E010C0953021F48A818093B40061C02F
:10025000963049F580ECF82E8B81813041F4E8E846
:10026000F0E002E1F093B200E093B10052C08230BE
:1002700021F4E6EFF0E007E3F5CF833009F049C061
:100280008A81882321F4E2EFF0E004E0EBCF8130B3
:1002900021F4EEECF0E004E2E5CF8230D1F5EAE9BA
:1002A000F0E004E3DFCF983019F4E6EBF0E008C0AB
:1002B000993021F48A818093B60009C09A3011F4F4
:1002C00001E0D0CF9B3031F48BE48093A2003093D7
:1002D00060001FC0913011F09330D9F48A818823D7
:1002E000C1F48C818138A9F4913011F48AE501C000
:1002F0008EE1809360008BE48093A2000AC0CE015F
:1003000050D3082F8F3F29F4888187FF1CC00E81AE
:100310001AC08F818823C1F48E818017A8F4082F1A
:1003200013C08091640087FD0FC0612FCE01EAD316
:100330000FEF801731F4009362008EE1809361002B
:1003400002C0811100E0FF24F0926400009362007B
:100350008091B300181614F41092B30080916100DC
:1003600084FF4FC0809162008F3F09F44AC0682F1C
:10037000893008F068E0861B809362001BE480915E
:10038000640080FD13EC8F5F80936400A8E9B0E007
:1003900087FF1BC0E091B100F091B200962F915001
:1003A00086FF07C09F3F59F084918D9331969150FD
:1003B000F9CF9F3F21F081918D939150FACFF09327
:1003C000B200E093B100772709C0662329F0CD0180
:1003D0004CD3682F772702C060E070E0C62F6930E9
:1003E00040F488E990E042D09C2F9C5FC83028F40C
:1003F00001C09EE18FEF809362001093970090936D
:1004000061009AE086B3837011F49150D9F7992373
:1004100039F49093B4009093AD008AE58093600026
:10042000DF91CF911F910F91FF90089589B780625E
:1004300089BF8BE48093A2000895A82FB92F8FEF76
:100440009FEF41E050EA615070F02D9138E0722F3B
:10045000782796958795269570FF02C08427952763
:100460003A95A9F7F0CF809590950895E6DF8D93A2
:100470009D930895CF93CFB7CF93B09BFECFB09B02
:100480000EC0B09B0CC0B09B0AC0B09B08C0B09B14
:1004900006C0C091B000C395C093B0009EC0DF936A
:1004A000C091AF00DD27C954DF4FB09B02C0DF9180
:1004B000E6CF2F930F931F9306B32FEF00FB20F986
:1004C0004F933F9316B34FEF012700FB21F93BE019
:1004D00031C04E7F012F16B3216028C0102F4D7FF1
:1004E0002260000006B329C04B7F2460012F00006A
:1004F00016B32BC016B3477F28602AC04F7E06B3C1
:1005000020612CC04F7D16B320622FC04F7B06B3F5
:10051000206432C0422706B349934FEF00001027F2
:1005200010FB20F916B31370A9F1297F91F201276E
:1005300000FB21F906B3237F89F23150F0F1102737
:1005400010FB22F916B3277E79F2012700FB23F96D
:100550002F7C81F206B3102710FB24F92F7971F25A
:1005600000C016B3012700FB25F92F7359F200C014
:1005700006B3102710FB26F9223040F200C016B354
:10058000012700FB27F9243028F64F77206816B39F
:100590000000F9CF3B503195333010E218BFB8F06E
:1005A000C31BD0400881033C51F10B3441F1198148
:1005B000412F1F772091AD00121731F40936A1F1B8
:1005C0000D3279F0013E69F022272093B5003F916A
:1005D0004F911F910F912F91DF91CF91CFBFCF916D
:1005E000189547FD0FEF0093B5003F914F911F9174
:1005F0000F912F91DF91C8B7C5FD3FCFEECF00918E
:10060000B500002321F31091B3001123A1F534307C
:10061000A2F13093B3000093AE001091AF003BE025
:10062000311B3093AF0029C00091B30001301CF59D
:100630000AE547FD09C03091610034FD20C00093F8
:100640006100C7E9D0E01FC03091600034FD17C0E1
:1006500000936000C2EAD0E016C0052710E008BB96
:100660001FC0052722C0052727C005272CC0052746
:1006700010E008BB33C04AE503C042ED01C0432F80
:10068000C4E1D0E032E017B31360C09A08B317BBDF
:100690005F9353E020E820FF052708BB27951795B7
:1006A0001C3FD8F620FF0527279508BB17951C3F50
:1006B000C0F620FF05272795179508BB1C3F98F625
:1006C00020FF0527279517951C3F08BB70F600C033
:1006D000499120FF052708BB279517951C3F38F641
:1006E00020FF0527279508BB17951C3F38F520FFED
:1006F00005272795179508BB1C3F10F520FF0527F8
:10070000279517951C3F08BBE8F4242F3A9519F656
:100710000C7F5F9108BB00C01091B400C651D0405F
:1007200011F01093AD0010E218BF016017B31C7FE9
:10073000402F4C7F08BB17BB48BB49CF0527D3CF01
:100740000527D8CF0527DDCF3091690031FD16C0D0
:1007500020918E00E22FFF27EE0FFF1FE359FF4F7E
:10076000918380832F5F2F703E7F80918D002817AB
:1007700009F4326020938E0030936900089520912F
:100780008D003091690030FF0CC021502F70E22F96
:10079000FF27EE0FFF1FE359FF4F0190F081E02D7F
:1007A00015C0E22FFF27EE0FFF1FE359FF4F2F5F0A
:1007B0000190F081E02D2F703D7F80918E00821797
:1007C00009F4316020938D0030936900CF010895C2
:1007D0008091680085FF04C011BA8FEF82BB089535
:1007E0008091670082BB80916C0080FF03C082B360
:1007F000809501C08FEF81BB0895EADF81E084BB63
:100800008EE385BB809168009BE08927880F880F65
:1008100088BB8CE387BB0895982F31B328B39D998B
:100820000CC0822F892388BB92FD02C08FEF81BB51
:1008300088E19D9907C08150E1F780916B0081604C
:1008400080936B0080B392FF31BB28BB992708953A
:10085000982F80916A008C7421F0892F992774DF7A
:100860000895909367008091680085FD07C092BB52
:1008700080916C0080FF02C0909591BB0895CF934A
:1008800090916A009570C82FC06C9111CF7D9091A6
:1008900068009C27C093680080916C0086FD04C0AE
:1008A00095FD96DF8BE0C827CC0FCC0FC8BB80919D
:1008B0006C0082FF03C0C095CC7FC7BBCF91089569
:1008C000282F887F85608093690022952695277060
:1008D00081E090E002C0880F991F2A95E2F7282F47
:1008E00080936A00332724FF02C08EEF01C08FEF90
:1008F00080936B0025703070232B41F0809168004D
:1009000085FF04C08F7D8093680062DF10928E00A7
:1009100010928D00089580916A008C7411F02FDF81
:1009200001C080B39927089593B3990F990F9760E9
:1009300080916C0086FD02C080E8982780916B0052
:100940009823892F9927089580916A008C7411F05B
:1009500088B301C086B3982F969596959F70809125
:100960006C0086FD02C08BE0982780916800807F34
:10097000982B892F99270895882329F09FE09A952D
:10098000F1F78150E1F70895982F80918F00882327
:1009900019F490939100A89A9093900090938F00EF
:1009A0000895FC018181809392006281738170932C
:1009B0009400609393004681578150939600409332
:1009C000950085E690E09093B2008093B10021817C
:1009D000222349F48281809365008381809366009D
:1009E00082E090E00895213089F48281882311F417
:1009F00092DF03C0813031F497DF8093650081E09E
:100A000090E00895823071F59FDFF7CF223059F4DE
:100A10008281882319F484811BDF24C0823011F580
:100A200084812DDF1FC08081803CA1F4822F815AF8
:100A30008330C0F4233A99F46630710581F4423072
:100A4000510569F489E397E390936600809365000C
:100A5000CA010895803431F4215A223018F48FEFFE
:100A600090E0089580E090E008951F93CF93DF9386
:100A7000FC01162FC0919300D0919400262F3327AC
:100A800080919500909196008217930710F4109131
:100A9000950080919200813A39F4812F9927AC0119
:100AA000BE01CF0144D217C0823A49F4812F992761
:100AB000DE0101971CF044D20192FBCF0CC0833AB7
:100AC00039F4812F9927AC01BE01CF0127D203C091
:100AD0002FEF30E012C0212F3327C20FD31FD09346
:100AE0009400C09393008091950090919600821B92
:100AF000930B9093960080939500C901DF91CF915D
:100B00001F910895FF920F931F93CF93DF93FC01E2
:100B1000F62EC0919300D0919400262F3327809118
:100B20009500909196008217930710F4F09095002D
:100B300080919200813A49F40F2D1127A801BF013D
:100B4000CE01F5D1C00FD11F10C0823A59F490E008
:100B50009F1558F48191DE01082EFAD1A8952196AF
:100B60009F5FF6CF2FEF30E010C0D0939400C0937A
:100B700093002F2D33278091950090919600821B32
:100B8000930B9093960080939500C901DF91CF91CC
:100B90001F910F91FF900895AF92BF92CF92DF9275
:100BA000EF92FF921F93CF93DF93CDB7DEB72897D5
:100BB0000FB6F894DEBF0FBECDBF7C01162F5E01CD
:100BC0000894A11CB11C6501662309F4EEC084E6FB
:100BD000DBDEF70181917F0184FF49C02FEF992768
:100BE00087FD9095A92FB92FFC017097E031F10591
:100BF000D0F5ED5EFF4F09948EDE27C095DE25C04F
:100C0000A3DE23C08FED01C087EF06DE1EC08091FA
:100C10006A008C7C19F42FEF30E025C087FF03C0F9
:100C200020E130E020C0ABDD282F33271CC08091AD
:100C30006A0087FF03C080E090E007C08FEF90E07C
:100C400004C0209169000FC081B3282F0CC024B3C9
:100C5000220F220F287F07C027B3269526952F70D5
:100C600002C020916C00F60121936F0196C01150D3
:100C700009F49BC021917F01992787FD9095A92FA9
:100C8000B92FFC01819708F088C0ED5DFF4F0994F2
:100C9000822FDEDD82C080916A0084FF07C020FDC4
:100CA00005C080916B008E7F80936B00922F96958C
:100CB000969580916C0086FD05C080E2982784B3EC
:100CC0008095982B9E7385B3817024C0822FD7DDC9
:100CD00064C022BB8BED02C022BB83EF9DDD5DC0F3
:100CE00080916A008C7409F458C0822F9927916012
:100CF0002BDD53C0822FE4DD50C021BB4EC0922FAC
:100D000096959695916C94BB80916C0086FD45C03C
:100D1000909585B3892B85BB40C0220F220F27BB3E
:100D20003CC0622F657480916C00862760936C00D4
:100D3000882399F1482F552740FF12C0262F3327CB
:100D4000C90180749070892B59F48091680085FDE9
:100D500007C020FF03C082B3809501C08FEF81BB25
:100D600042FF0FC0262F3327C90180749070892B52
:100D700041F422FF04C088B380958C7301C08CE3DA
:100D800087BB46FF0AC0862F992780749070892BF5
:100D900021F433DD02C0822FEFDD115009F019CFAD
:100DA0006C2D6A1911F0C501DDD928960FB6F8949B
:100DB000DEBF0FBECDBFDF91CF911F91FF90EF90AF
:100DC000DF90CF90BF90AF900895CFE5D4E0DEBF25
:100DD000CDBF10E094B714BF479A85B7806885BF30
:100DE00093FF0BC086B3992783709070892B29F0ED
:100DF00085B78F78806285BF889518DB7894ABEFD4
:100E0000BFEF9ED0802D992780936C008F3F11F407
:100E100010926C00109267008CEC80936800EDDCFF
:100E200080E24EDDC0916A008C2F992782FF0CC0B2
:100E30008091690080FD3DC09D993BC0A0DC82BBD4
:100E4000C29881E099DD2CC083FF2CC0809168009E
:100E500085FF12C08091690081FD2BC0C39903C03A
:100E60009C9927C0C39A9C9B24C080B399279D99C5
:100E700091606ADCC3981DC0C29B10C0809169005C
:100E800080FD17C09D9915C07ADC82BB28B32473FE
:100E90008070892B09F0286028BBC2989D9B09C0EF
:100EA000C29A07C086B3992783709070892B09F086
:100EB0008895C091B0001C1731F486B399278370D0
:100EC0009070892B09F4A89574D91C1709F4AACF3E
:100ED0001C2F20918F00222389F080919100815056
:100EE00031F485B391E0892785BB80919000215032
:100EF00009F4A89820938F0080939100E19992CFF4
:100F0000ABEFBFEF1DD0802D90916C00891709F4D5
:100F100089CFABEFBFEF092E1BD084CFFB01DC01E3
:100F200002C005900D9241505040D8F70895FB0142
:100F3000DC0102C001900D9241505040D8F7089555
:100F4000E199FECFBFBBAEBBE09A11960DB20895FA
:100F5000E199FECFBFBBAEBB0DBA11960FB6F894A8
:080F6000E29AE19A0FBE089528
:040F68005A5AFF00D2
:00000001FF
